:020000040000FA
:040000006E303A28FC
:08000800A000030EA100831209
:1000100005191028831601178312B23081002B288E
:1000200083160113831203140B190310A80DA90DD5
:10003000AA0DAB0DAC0DAC16FF302C02031D2B2806
:10004000FA302B02031D2B2831152A08AF0029088E
:10005000AE002808AD008B100B11210E8300A00EFE
:04006000200E090065
:0C007400203084008001840A6030040207
:10008000031C3C281230B0008C2183160C308505EF
:1000900087018312850187010730990000309A009B
:1000A000103083168E008312603083168F00831207
:1000B0000030831691008312C830831681008312AA
:1000C00031309000003083168C00831210308B008A
:1000D000831600309B001C141A088312BC00831680
:1000E00010309B001C141A088312BD00A521810149
:1000F0008E018F010B118B100B108C018B178F2031
:10010000311992206E21B30B8D2803108519031429
:10011000B90DF030390203191721A6217F28640098
:100120003210080031110130B7008B13203037072F
:1001300083169B001C141A088312A4001030370782
:1001400083169B001C141A088312A300A600023019
:10015000A6060030370783169B001C141A0883126A
:10016000A200A7000130A7068B17321CBD28220968
:100170000339A200A309A409A50924082F02031D1D
:10018000112923082E02031D112922082D02031D07
:10019000112901303702031DD2283D18D2283D1401
:1001A0003E148D2102303702031DDB28BD18DB28E9
:1001B000BD143E14902103303702031DE4283D197D
:1001C000E4283D153E14932104303702031DED2829
:1001D000BD19ED28BD153E14962105303702031DCB
:1001E000F6283D1AF6283D163E14992106303702AE
:1001F000031DFF28BD1AFF28BD163E149C210730A1
:100200003702031D08293D1B08293D173E149F2175
:1002100008303702031D1129BD1B1129BD173E14DB
:10022000A221B70A093037020318080095280130C7
:10023000B600B300B400B500B70085018701B11363
:100240008F20B30B3D29031085190314B90DF0302D
:10025000390203196429B41F8501B41F8701B40B47
:100260003D293708B6080319B60003193B29FF30AA
:1002700085008700B6039630B400311D2029311166
:10028000321C47292D090339AD00AE09AF092F1CD7
:1002900020298E018F010C1C20290C102E1E2029D4
:1002A0008B1320303707BB002F08BA00772110309E
:1002B0003707BB002E08BA00772100303707BB0094
:1002C0002D08BA0077218B1785018701B70AB6017F
:1002D00009303702031C2029A52108003E1C080014
:1002E0003E101030BB003D08BA00772108008B1388
:1002F0003A0883161C159A0083123B0883169B004C
:1003000055309D00AA309D009C1464009C188529DE
:100310001C1183128B17080008000130BD00080073
:100320000230BD0008000430BD0008000830BD00E8
:1003300008001030BD0008002030BD00080040302B
:10034000BD0008008030BD00080008008F080319B8
:1003500008008F0107303D0503199E2A02303D0534
:10036000031D51105408EB3C031805125118BB290A
:10037000D40BC629C029D4035408C83C031CC62981
:100380000516F530D4005108013AD10002303D0580
:10039000031DD1105508E63C03188512D118D32946
:1003A000D50BDE29D829D5035508B93C031CDE2915
:1003B0008516F030D5005108023AD10002303D05D3
:1003C000031D51115608DC3C031805105119EB2987
:1003D000D60BF629F029D6035608B63C031CF6299D
:1003E0000514E630D6005108043AD10002303D052C
:1003F000031DD1115708F03C03188510D119032AA9
:10040000D70B0E2A082AD7035708D73C031C0E2AFD
:100410008514FA30D7005108083AD10002303D0562
:10042000031D51125808E03C03188710511A1B2A6B
:10043000D80B262A202AD8035808C13C031C262A98
:100440008714EA30D8005108103AD10006303D0533
:10045000031DD1125908D43C03180711D11A332AAD
:10046000D90B3E2A382AD9035908A73C031C3E2A37
:100470000715DE30D9005108203AD10006303D057D
:10048000031D51135A08BF3C03180710511B4B2A78
:10049000DA0B562A502ADA035A089C3C031C562AC7
:1004A0000714C930DA005108403AD10006303D0542
:1004B000031DD1135B08D73C03188712D11B632A95
:1004C000DB0B6E2A682ADB035B08BE3C031C6E2A2A
:1004D0008716E130DB005108803AD10006303D0537
:1004E000031D52105C08F13C0318071252187B2AB6
:1004F000DC0B862A802ADC035C08CF3C031C862A9E
:100500000716FB30DC005208013AD20006303D05E8
:10051000031DD2105D08E93C03188711D218932AF5
:10052000DD0B9E2A982ADD035D08B23C031C9E2A3F
:100530008715F330DD005208023AD20018303D052D
:100540000319EE2ABD1DAA2A54083C3C031CAA2A02
:1005500085018701D40B0800D0034630D4000B304E
:100560005002031DB42A05160A305002031DB92A91
:10057000851609305002031DBE2A051408305002AA
:10058000031DC32A851407305002031DC82A87148F
:1005900006305002031DCD2A071505305002031DF9
:1005A000D22A071404305002031DD72A87160330BD
:1005B0005002031DDC2A071602305002031DE12AF7
:1005C000871501305002031DE52A12305002031C2A
:1005D0000800850187010C30D000080020303D055F
:1005E0000319382BD40BF92A0508103A85008230FC
:1005F000D400D50B002B0508203A85007D30D500AE
:10060000D60B072B0508013A85007330D600D70BAF
:100610000E2B0508023A85008730D700D80B152B22
:100620000708023A87007730D800D90B1C2B07083F
:10063000043A87006B30D900DA0B232B0708013A04
:1006400087005630DA00DB0B2A2B0708203A870098
:100650006E30DB00DC0B312B0708103A8700883046
:10066000DC00DD0B382B0708083A87008030DD00FE
:1006700040303D050319AF2B5408E63C0318051222
:10068000D40B5E2B0516F030D4002130DE070318A2
:100690005C2BB130D507FA30D607C830D7076430A5
:1006A000D8079630D907BE30DA07AA30DB079A3070
:1006B000DC07C430DD075E2B8030BD005508823C6E
:1006C00003188512D50B672B85168C30D50056087C
:1006D000653C03180510D60B702B05146F30D6003F
:1006E0005708913C03188510D70B792B85149B3044
:1006F000D7005808D73C03188710D80B822B8714D3
:10070000E130D8005908503C03180711D90B8B2B46
:1007100007155A30D9005A08873C03180710DA0B1E
:10072000942B07149130DA005B08BD3C0318871244
:10073000DB0B9D2B8716C730DB005C08703C031871
:100740000712DC0BA62B07167A30DC005D08A73CED
:1007500003188711DD0BAF2B8715B130DD0080301A
:0E0760003D050319B62B85018701DE01080057
:084000000B00030002000600A2
:02400E00CC33B1
:10420000010078007A007C007E007B0079007F004E
:104210007D007A0078007E007C00FF00FF00FF0038
:104220000000F200F600FA00FE00F200F600FA00CC
:10423000FE00F200F600FA00FE00FF00FF00FF00A3
:10424000010005000500050005000900090009003E
:1042500009000D000D000D000D00FF00FF00FF0024
:10426000FF00FF00FF00FF00FF00FF00FF00FF0056
:10427000FF00FF00FF00FF00FF00FF00FF00FF0046
:10428000FF00FF00FF00FF00FF00FF00FF00FF0036
:10429000FF00FF00FF00FF00FF00FF00FF00FF0026
:1042A000FF00FF00FF00FF00FF00FF00FF00FF0016
:1042B000FF00FF00FF00FF00FF00FF00FF00FF0006
:1042C000FF00FF00FF00FF00FF00FF00FF00FF00F6
:1042D000FF00FF00FF00FF00FF00FF00FF00FF00E6
:1042E000FF00FF00FF00FF00FF00FF00FF00FF00D6
:1042F000FF00FF00FF00FF00FF00FF00FF00DD00E8
:00000001FF
